:10000000F32210309307B0001305200573000000A1
:100010001305600573000000130530037300000032
:1000200013052003730000001303001033F3620074
:100030009307B00013059004B3D7670E7300000058
:100040001303000133F362009307B000130550045B
:10005000B3D7670E730000003713000033F362005C
:100060009307B0001305D004B3D7670E73000000E8
:100070001303100033F362009307B000130510045C
:10008000B3D7670E730000001303000233F362005E
:100090009307B00013056004B3D7670E7300000028
:1000A0001303800033F362009307B000130540048C
:1000B000B3D7670E730000003703010033F362000B
:1000C0009307B00013051005B3D7670E7300000047
:1000D000371300001303038033F362009307B0006B
:1000E0001305C004B3D7670E73000000130340006C
:1000F00033F362009307B00013053004B3D7670EE3
:10010000730000001303200033F362009307B00074
:1001100013052004B3D7670E7300000013030020FB
:1001200033F362009307B0001305A004B3D7670E42
:10013000730000003703080033F362009307B00038
:1001400013054005B3D7670E730000003783000026
:1001500033F362009307B00013050005B3D7670EB1
:10016000730000003703200033F362009307B000F0
:1001700013056005B3D7670E730000001303000872
:1001800033F362009307B00013058004B3D7670E02
:10019000730000003703040033F362009307B000DC
:1001A00013053005B3D7670E730000009307A00056
:0401B00073000000D8
:00000001FF
